:100000000C94B4020C94E5020C94E5020C94E50205
:100010000C94E5020C94E5020C94E5020C94E502C4
:100020000C94E5020C94E5020C94E5020C94E502B4
:100030000C94E5020C94E5020C94E5020C94E502A4
:100040000C94E5020C94E5020C94E5020C94E50294
:100050000C94E5020C94E5020C94E5020C94C01B90
:100060000C94E5020C948A1B0C94601B0C94E50222
:100070000C94E5020C94E5020C94E5020C94E50264
:100080000C94E5020C94E5020C94E5020C94E50254
:100090000C94E5020C94E5020C94E5020C940A1C05
:1000A0000C94E5020C94E5020C94E5020C94E50234
:1000B0000C94E5020C94E5020C94E5020C94E50224
:1000C0000C94E5020C94E5020C94E5020C94E50214
:1000D0000C94E5020C94E5020C94E5020C94E50204
:1000E0000C94E502084AD73B3BCE016E84BCBFFDB1
:1000F000C12F3D6C74319ABD56833DDA3D00C77FF8
:1001000011BED9E4BB4C3E916BAAAABE0000008090
:100110003F07634236B79BD8A71A39685618AEBA5C
:10012000AB558C1D3CB7CC5763BD6DEDFD753EF6F0
:10013000177231BF000000803F08000000BE92240B
:1001400049123EABAAAA2ABECDCCCC4C3E00000040
:1001500080BEABAAAAAA3E00000000BF000000803B
:100160003F0000000000084178D3BB4387D1133D16
:10017000190E3CC3BD4282AD2B3E68EC8276BED9DF
:100180008FE1A93E4C80EFFFBE01C4FF7F3F00001E
:10019000000000000C94EB240C9417030C94EB0863
:1001A0000C94FA080C94450C0C944F100C94930387
:1001B0000C9418040C94AE060C949C040C94A204A9
:1001C0000C94BA040C9462030C94AF060C94910442
:1001D0000C94B6060C941A030C942E1D0C94C704B0
:1001E0000C9402100C94E7020C948D040C94A60459
:1001F0000C94EA080C9499040C94AC040C948503B8
:100200000C94C8040C94CB030C9471030C94180345
:100210000C9487040C9468090C94C2040C9427096C
:100220000C9495040C94BE040C94B0040C94CC046F
:100230000C94B4044E414E494E495459494E46CD52
:10024000CCCC3D0AD7233C17B7D13877CC2B32958D
:1002500095E6241FB14F0A000020410000C842006B
:10026000401C4620BCBE4CCA1B0E5AAEC59D740035
:10027000407A10F35A00A0724E18090010A5D4E875
:100280000000E87648170000E40B54020000CA9A08
:100290003B000000E1F5050000809698000000405A
:1002A000420F000000A0860100000010270000009F
:1002B00000E803000000006400000000000A0000E5
:1002C0000000000100000000002C76D888DC674F99
:1002D0000823DFC1DFAE59E1B1B796E5E3E453C6C9
:1002E0003AE651997696E8E6C28426EB898C9B62C1
:1002F000ED407C6FFCEFBC9C9F40F2BAA56FA5F46B
:1003000090055A2AF75C936B6CF9676DC11BFCE092
:10031000E40D47FEF520E6B500D0ED902E030094E5
:100320003577050080841E080000204E0A0000007A
:10033000C80C333333330F986E12831141EF8D2184
:1003400014893BE65516CFFEE6DB18D1844B381BEB
:10035000F77C1D901DA4BBE424203284725E2281B0
:1003600000C9F124ECA1E53D273E6128782C792CC9
:100370007A292F673A00543D00495220466C616D3E
:1003800065204C6576656C3D00476173206C657631
:10039000656C3D0023496E76616C6964206B6579FC
:1003A00021003E482D6669656C643A2028000000F3
:1003B0002100240027002A002D0030003300010115
:1003C0000000040107010A010000220025002800A6
:1003D0002B002E003100340002010000050108014D
:1003E0000B0123626D70206661696C6564002357A0
:1003F000656C636F6D6520746F20757365204E6149
:100400006E6F204C6F67676572004D533D00234E41
:100410006F2055562073656E736F722100503D003A
:1004200042543D004448543D002344757261746950
:100430006F6E3D0054494D45443D0023496E74653F
:100440007276616C3D0054494D45493D0053484F1B
:1004500057533D004C6F67676572204E616D653A7A
:1004600020004C4F474745520056455253494F4E86
:10047000005245424F4F5400000020002300260048
:1004800029002C002F0032000001000003010601AA
:10049000090105050505070508080808020202020A
:1004A0000A0A080804040404010101010101010110
:1004B0000303030303030303040707070C0C0C0CDB
:1004C0000C0C0C0C020202020606060606060606C4
:1004D0000B0B0B0B0B0B0B0B010210202008081051
:1004E00020401020408002010201080402010102A4
:1004F000040810204080804020100804020180047D
:1005000002018040201008040201080402010102D7
:1005100004081020408001020408102040800000E0
:100520000A0B02090C0D0E0807030401000000006D
:1005300000000000000000000000000000000000BB
:100540000000000000000000000012111000000078
:10055000000000000000000000000000000000009B
:10056000000000002E1DEB2411241FBECFEFD1E2AE
:10057000DEBFCDBF00E00CBF13E0A0E0B2E0E6E5D7
:10058000F2E600E00BBF02C007900D92A631B10762
:10059000D9F725E0A6E1B3E001C01D92A036B2076D
:1005A000E1F712E0C3EBD2E000E006C021970109B9
:1005B000802FFE010E94D62EC23BD10780E00807A3
:1005C000A9F70E94141E0C9419310C94000090910C
:1005D0009803809197032FEF3FEF981748F4E92F86
:1005E000F0E0E958FC4F208130E09F5F9093980342
:1005F000C901089590919803809197032FEF3FEFE1
:10060000981748F4E92FF0E0E958FC4F208130E0DA
:100610009F5F90939803C901089591E09093C5035B
:100620008093E7031092C6031092E803089508959B
:1006300008950895AF92BF92CF92DF92EF92FF920A
:100640000F931F93CF93DF936C017B018B01040FFA
:10065000151FEB015E01AE18BF08C017D10759F096
:100660006991D601ED91FC910190F081E02DC601D8
:100670001995892B79F7C501DF91CF911F910F91C2
:10068000FF90EF90DF90CF90BF90AF900895FC0166
:10069000448155816081718189EE93E00C941A0345
:1006A000CF93DF930E944703EC0142E050E06EE4F9
:1006B00072E089EE93E00E941A038C0F9D1FDF9178
:1006C000CF910895FC01538D448D252F30E0842F68
:1006D00090E0821B930B541710F0CF96089501976A
:1006E0000895FC01918D828D981761F0A28DAE0F57
:1006F000BF2FB11D5D968C91928D9F5F9F73928FDE
:1007000090E008958FEF9FEF0895FC01918D828D09
:10071000981731F0828DE80FF11D858D90E00895D6
:100720008FEF9FEF0895FC01918D228D892F90E02E
:10073000805C9F4F821B91098F739927089589EEE2
:1007400093E00E94930321E0892B09F420E0822F9B
:100750000895FC01A48DA80FB92FB11DA35ABF4F56
:100760002C91848D90E001968F739927848FA689B0
:10077000B7892C93A089B1898C91837080648C9304
:10078000938D848D981306C00288F389E02D8081B3
:100790008F7D80830895EF92FF920F931F93CF93E5
:1007A000DF93EC0181E0888F9B8D8C8D98131AC0AC
:1007B000E889F989808185FF15C09FB7F894EE8993
:1007C000FF896083E889F9898081837080648083F0
:1007D0009FBF81E090E0DF91CF911F910F91FF903B
:1007E000EF900895F62E0B8D10E00F5F1F4F0F73E3
:1007F0001127E02E8C8D8E110CC00FB607FCFACF9E
:10080000E889F989808185FFF5CFCE010E94A9038F
:10081000F1CFEB8DEC0FFD2FF11DE35AFF4FF0826E
:100820009FB7F8940B8FEA89FB8980818062CFCFD4
:10083000CF93DF93EC01888D8823B9F0AA89BB8917
:10084000E889F9898C9185FD03C0808186FD0DC002
:100850000FB607FCF7CF8C9185FFF2CF808185FF23
:10086000EDCFCE010E94A903E9CFDF91CF9108958A
:1008700080E090E0892B29F00E949F0381110E9463
:10088000000080E090E0892B49F080E090E0892B27
:1008900029F00E94000081110E94000080E090E099
:1008A000892B49F080E090E0892B29F00E9400001C
:1008B00081110E94000080E090E0892B49F080E0E7
:1008C00090E0892B29F00E94000081110C94000017
:1008D00008958150823108F05AC0E82FF0E088274F
:1008E000EB58FB4F8F4F0C94D62E95049904870438
:1008F0008D049104C7049C04A204A604AC04B004B3
:10090000B404BA04BE04C704C204C804CC04809171
:1009100080008F77809380000895809180008F7D84
:10092000F9CF80918000877FF5CF84B58F7784BD24
:10093000089584B58F7DFBCF8091B0008F77809331
:10094000B00008958091B0008F7DF9CF8091900024
:100950008F77809390000895809190008F7DF9CFDC
:1009600080919000877FF5CF8091A0008F77809352
:10097000A00008958091A0008F7DF9CF8091A00004
:10098000877FF5CF809120018F7780932001089594
:10099000809120018F7DF9CF80912001877FF5CF55
:1009A000CF93DF93E5E5F5E08491EFE0F5E0D491B6
:1009B000E9ECF4E0C491CC23A1F081110E94690418
:1009C000EC2FF0E0EE0FFF1FE858FB4FA591B4911C
:1009D000EC91ED2381E090E009F480E0DF91CF918C
:1009E000089580E090E0FACF1F93CF93DF93282FF4
:1009F00030E0F901E25EFA4F8491F901E852FB4FD1
:100A0000D491F901EE56FB4FC491CC23A9F0162FD7
:100A100081110E946904EC2FF0E0EE0FFF1FE853F4
:100A2000FC4FA591B4918FB7F894EC91111108C0C7
:100A3000D095DE23DC938FBFDF91CF911F91089576
:100A4000DE2BF8CFCF93DF9390E0FC01E852FB4F11
:100A500024918E569B4FFC0184918823D1F090E025
:100A6000880F991FFC01E255FC4FA591B491FC0140
:100A7000E853FC4FC591D49161110EC09FB7F89413
:100A80008C91E22FE0958E238C932881E223E883DA
:100A90009FBFDF91CF9108958FB7F894EC91E22B2F
:100AA000EC938FBFF6CF3FB7F8948091630390919A
:100AB0006403A0916503B091660326B5A89B05C0A9
:100AC0002F3F19F00196A11DB11D3FBFBA2FA92FCD
:100AD000982F8827BC01CD01620F711D811D911DCA
:100AE00042E0660F771F881F991F4A95D1F7089536
:100AF0008F929F92AF92BF92CF92DF92EF92FF922E
:100B00006B017C010E9453054B015C01C114D104AF
:100B1000E104F104B9F00E945305681979098A09C2
:100B20009B09683E73408105910580F321E0C21A5C
:100B3000D108E108F10888EE880E83E0981EA11C18
:100B4000B11CE4CFFF90EF90DF90CF90BF90AF90BB
:100B50009F908F9008958F929F92AF92BF92EF9245
:100B6000FF921F93CF93DF93C82F109254051092DA
:100B7000550510925605109257051092580561E0E0
:100B800087E30E94220560E087E30E94F4046C2F53
:100B900070E090E080E00E94780560E087E30E94CA
:100BA00022058BE990E00197F1F7C0E9D1E00E94BE
:100BB000D004892B71F42197D1F78EEF9FEFDF914D
:100BC000CF911F91FF90EF90BF90AF909F908F902B
:100BD0000895C0E9D1E00E94D004019719F421974B
:100BE000D1F7EBCFD8E2C0E810E090E9E92EFF247E
:100BF000F3940E94D004892B29F481E0E81AF108CB
:100C0000C1F7DBCF0E9453054B015C0180E9E82E60
:100C1000FF24F3940E94D004019729F481E0E81A9C
:100C2000F108C1F7CACF0E945305681979098A09EA
:100C30009B09693271058105910538F0E12FF0E0DB
:100C4000E45BFA4F80858C2B8087C69511F41F5F7B
:100C5000C0E8D15051F690E080E0B1CF8F929F92E2
:100C6000AF92BF92CF92DF92EF92FF920F931F93BA
:100C7000CF93DF938AE0882E912CD0E0C0E0CC2483
:100C8000CA9493E0D92EEE24EA9423E0F22EB12CFC
:100C9000A12C10E000E080917B00877F80937B0097
:100CA0008091150220E4829FC0011124816080930D
:100CB0007C0080917A00806480937A0080917A0031
:100CC00086FDFCCF90917800809179008927982744
:100CD00089270817190790F1A816B90608F45C01CE
:100CE0008E159F0568F18C159D0508F46C01C80FE1
:100CF000D91F65E070E080E090E00E94780581E017
:100D0000881A910841F60A0D1B1DCE01801B910B1C
:100D10008C199D098E199F0966E070E00E94C22E11
:100D2000CB01DF91CF911F910F91FF90EF90DF905A
:100D3000CF90BF90AF909F908F9008958C01D0CFAF
:100D40007C01D5CF2FB7F89460915F037091600359
:100D500080916103909162032FBF0895089580915F
:100D6000970390919803891B990B089508952091FA
:100D70003B03260F3327331F21323105ECF420913A
:100D8000BF03FC0190E080E0243069F082E0089528
:100D9000A0913B032191AC01455E5C4FA40FB52FA0
:100DA000B11D2C930196861798F380913B03680F31
:100DB00060933B0380E0089581E008951092BF03A3
:100DC00081E08093BE031092990361E084E10E9468
:100DD000F40461E085E10E94F404E9EBF0E0808135
:100DE0008E7F808380818D7F808388E48093B800AC
:100DF00085E48093BC0008951092980310929703A5
:100E00001092C6031092E8030E94DE0687E193E089
:100E1000909376038093750388E193E09093740335
:100E2000809373030895CF93DF9391E090931A0317
:100E30008823B9F0C091B800D091BA008091BC006D
:100E40008A7B8093BC0060E084E10E94F40460E04F
:100E500085E10E94F4040E94DE06D093BA00C0939C
:100E6000B800DF91CF910895CF92DF92EF92FF9279
:100E70000F931F93CF93DF93D091E80381E0D1329A
:100E800008F09CC0C091E7030E9453056B017C01F0
:100E90008091BF0381116CC082E08093BF0381E029
:100EA0008093BE038FEF8093BD031092BC03D09359
:100EB000BB03A7ECB3E0EBE9F3E080E0D8138DC00F
:100EC00010929A0380919A03CC0FC82BC0939A0377
:100ED00080919903813009F084C0109299030E9497
:100EE00053056B017C0180919A038093BB00809134
:100EF000C1039091C203A091C303B091C403892B95
:100F00008A2B8B2BA1F00E9453050091C1031091F5
:100F1000C2032091C3033091C4036C197D098E096B
:100F20009F09061717072807390708F442C0809160
:100F3000BC0083FDD8CF85EC8093BC000E94530594
:100F40006B017C018091BF03823009F44CC0809119
:100F5000BD038F3F09F469C08091BD03803209F45D
:100F600066C08091BD03803309F463C084E026C06D
:100F70008091C1039091C203A091C303B091C403B7
:100F8000892B8A2B8B2B09F483CF0E945305009168
:100F9000C1031091C2032091C3033091C4036C19A3
:100FA0007D098E099F09061717072807390708F0DA
:100FB0006FCF8091C0030E94130785E01092C60393
:100FC0001092E8031092C503DF91CF911F910F910A
:100FD000FF90EF90DF90CF9008959D9191938F5F58
:100FE0006DCF85EEA9CF8091C1039091C203A091EE
:100FF000C303B091C403892B8A2B8B2B09F4A2CF96
:101000000E9453050091C1031091C2032091C303B4
:101010003091C4036C197D098E099F0906171707C3
:101020002807390708F08ECFC4CF80E0C7CF82E011
:10103000C5CF83E0C3CFCF92DF92EF92FF920F93A1
:101040001F93CF93DF93D82FC62F613208F098C03B
:101050000E9453056B017C018091BF0381116BC01D
:1010600081E08093BF038093BE039FEF9093BD0305
:101070001092BC039C0F9093BB0380939A038091C2
:101080009A03DD0FD82BD0939A0380919903813076
:1010900009F078C0109299030E9453056B017C01FE
:1010A00080919A038093BB008091C1039091C20309
:1010B000A091C303B091C403892B8A2B8B2BA1F081
:1010C0000E9453050091C1031091C2032091C303F4
:1010D0003091C4036C197D098E099F090617170703
:1010E0002807390708F448C08091BC0083FDD8CF99
:1010F00085EC8093BC000E9453056B017C018091BC
:10110000BF03813009F440C08091BC038C1710F4F8
:10111000C091BC03EBE9F3E0A7E7B3E080E08C13F8
:1011200055C08C2FDF91CF911F910F91FF90EF90C1
:10113000DF90CF9008958091C1039091C203A09158
:10114000C303B091C403892B8A2B8B2B09F484CF62
:101150000E9453050091C1031091C2032091C30363
:101160003091C4036C197D098E099F090617170772
:101170002807390708F070CF8091C0030E94130739
:10118000C0E0CFCF85EEB5CF8091C1039091C2036F
:10119000A091C303B091C403892B8A2B8B2B09F434
:1011A000AECF0E9453050091C1031091C20320915C
:1011B000C3033091C4036C197D098E099F0906177A
:1011C00017072807390708F09ACFD6CF91919D933A
:1011D0008F5FA5CF0895E091980380919703E8175A
:1011E00030F4F0E0E958FC4F808190E008958FEFF3
:1011F0009FEF0895CF92DF92EF92FF920F931F938C
:10120000CF93DF937C01CB018A012091C503222378
:1012100089F0EB016B01C40ED51ECC15DD0569F01C
:101220006991D701ED91FC910190F081E02DC7010A
:101230001995F3CF642F0E94B706C801DF91CF91B3
:101240001F910F91FF90EF90DF90CF900895CF9373
:10125000DF931F92CDB7DEB769832091C5032223A8
:10126000F9F02091E803203258F021E030E0FC0151
:101270003383228390E080E00F90DF91CF91089537
:101280008091C603E82FF0E0E953FC4F99819083E9
:101290008F5F8093C6038093E80381E090E0ECCFFA
:1012A00061E0CE0101960E94B706F7CFCF93C82F19
:1012B00083E50E940D036DE286E894E00E94270911
:1012C0006C2F86E894E00E942709CF910C94340794
:1012D00090E080E00895FC0124813581232B41F0CA
:1012E0000E94470369E170E080E090E00C9478058B
:1012F00008950E941B081092980380939703089505
:10130000CF93C82F87E70E940D036C2F86E894E0E7
:101310000E9427090E94340787E70E940D0361E0BD
:1013200070E087E790E00E9479090E94FA02C82FD6
:101330000E9434078C2FCF910895CF93DF93C82F4D
:1013400087E70E940D036C2F86E894E00E9427092E
:101350000E94340787E70E940D0362E070E087E790
:1013600090E00E9479090E94FA02D82F80E0C82FED
:101370000E94FA02C82BD92B0E943407CE01DF91BC
:10138000CF91089587E70E940D0364EF86E894E00B
:101390000E9427096EE286E894E00E9427090E94D5
:1013A000340765E070E080E090E00E94780586EF09
:1013B0000C949D094F925F926F927F928F929F92B1
:1013C000AF92BF92CF92DF92EF92FF92CF93DF93D3
:1013D00000D01F921F92CDB7DEB70E94C2094C0108
:1013E000B12CA12C209121052295220F220F207CC7
:1013F0002C5C298387E70E940D0364EF86E894E064
:101400000E942709698186E894E00E9427090E94CA
:10141000340780912105811174C165E070E080E09E
:1014200090E00E94780586EF0E949D09B0E0A0E060
:10143000CC24D82EE92EFA2E88EF0E948009A7012D
:101440009601282B29833A834B835C8330912105B5
:101450003D838091360590913705A5019401281BA5
:10146000390B41095109A0913405B09135050E940D
:10147000072B4B015C01AFE0B594A7949794879438
:10148000AA95D1F760912E0570912F05072E000CBB
:10149000880B990BBBE0660F771F881F991FBA95C1
:1014A000D1F72091300530913105032E000C440B0B
:1014B000550B280D391D4A1D5B1D0E94E82A820E1E
:1014C000931EA41EB51E7501640140EAC41A4FE0C4
:1014D000D40AE108F108A7019601C701B6010E94EC
:1014E000B22E4B015C018CE0B594A794979487943D
:1014F0008A95D1F7A0912605B09127050E94122B5D
:101500002B013C019DE075946794579447949A95FC
:10151000D1F7A0912805B0912905A50194010E9459
:10152000122B9C01552737FD5095452F240D351D55
:10153000461D571D2E5F3F4F4F4F5F4F62E0559541
:101540004795379527956A95D1F730584F4F5F4F9C
:10155000A0913205B09133050E94072B2B013C016D
:101560007FE076946794579447947A95D1F788E012
:1015700090E05D81851B910929813A814B815C81D5
:1015800004C056954795379527958A95D2F72983B4
:101590003A834B835C83A0912A05B0912B05A5016A
:1015A00094010E94122B4B015C01EBE0B594A794CF
:1015B00097948794EA95D1F7A0912405B0912505D9
:1015C000A70196010E94122BFBE0959587957795D0
:1015D0006795FA95D1F7680D791D8A1D9B1D80903E
:1015E000220590902305092C000CAA08BB08A2E054
:1015F000880C991CAA1CBB1CAA95D1F7680D791DF3
:101600008A1D9B1D0D8004C0660F771F881F991FC0
:101610000A94D2F76E5F7F4F8F4F9F4F24E030E0E8
:1016200040E050E00E94E82A89819A81AB81BC8128
:10163000821B930BA40BB50B9C01AD0160E573EC11
:1016400080E090E00D8004C096958795779567952A
:101650000A94D2F70E94B22E97FD66C0660F771FDC
:10166000881F991FA30192010E941A2B69017A0118
:101670009927F7FC9A958F2D7E2D6D2D9B01AC013E
:101680000E94B22E9B01AC01AEEDBBE00E94072B85
:101690004B015C01A3E4B3EEA70196010E94152B58
:1016A000BC01992777FD9095892F4501BB2497FCB4
:1016B000B094AB2C680D791D8A1D9B1D6153714F31
:1016C0008F4F9F4F44E095958795779567954A95FD
:1016D000D1F76C0D7D1D8E1D9F1D0F900F900F90EB
:1016E0000F900F90DF91CF91FF90EF90DF90CF9010
:1016F000BF90AF909F908F907F906F905F904F9032
:101700000895813029F468E070E080E090E089CEAF
:10171000823029F46EE070E080E090E082CE6AE1F1
:1017200070E080E090E07DCEA30192010E941A2B30
:1017300069017A01CC0CDD1CEE1CFF1C99CFAF9225
:10174000BF92DF92EF92FF920F931F93CF93DF939D
:101750005C0102E914E0D0E0C0E0F801D1908F0113
:101760007501EC0EFD1EC7010E94D22AD81621F089
:101770006D2DC7010E94DA2A2196CC34D10569F774
:1017800082E994E0DF91CF911F910F91FF90EF904C
:10179000DF90BF90AF900895FC0180819181009708
:1017A00011F00C94292560E070E0CB010895FB0155
:1017B00044815581FC01248135812417350778F057
:1017C00080819181009759F0FB01608171816115E1
:1017D000710529F00E94FC3021E0892B09F020E0FE
:1017E000822F08950F931F93CF93DF938C01EB010A
:1017F000FC01808191810097E1F068817981611518
:101800007105A9F0428153812C813D814217530714
:1018100070F00E94F5308C819D81F801958384835E
:101820001D821C82DF91CF911F910F9108950E941C
:101830007A2F88819981F801918380838A819B81A5
:10184000938382838C819D819583848319821882FE
:101850001B821A82E5CFCF93DF93EC0188819981B7
:10186000009711F00E947A2F198218821D821C8223
:101870001B821A82DF91CF910895FC0180819181B2
:10188000009711F00C947A2F08950C947A2F0F93EF
:101890001F93CF93DF93EC0188819981009759F0D2
:1018A0002A813B812617370730F081E0DF91CF9105
:1018B0001F910F9108958B016F5F7F4F0E9403303E
:1018C000009759F0998388831B830A832C813D817B
:1018D000232B59F7FC011082E8CF80E0E7CFEF928D
:1018E000FF920F931F93CF93DF936115710541F41E
:1018F00080E0DF91CF911F910F91FF90EF900895BD
:1019000041155105B1F07B01EC010C811D81040FE3
:10191000151FB8010E94470C882351F32881398193
:101920008C819D81B701820F931F0E94F5301D832A
:101930000C8381E0DECFCF93DF93EC01FB010190BC
:101940000020E9F73197AF01461B570B0E946F0C3F
:10195000811103C0CE010E942B0CCE01DF91CF91EB
:101960000895CF93DF93EC01FB01448155816081A1
:1019700071810E946F0C811103C0CE010E942B0C5B
:10198000CE01DF91CF910895FB01448155816081A3
:1019900071810C946F0CEF92FF920F931F93CF9372
:1019A000DF93EC018B01CB010E9457257C01BC0128
:1019B000CE010E94470C81110BC0CE010E942B0C5E
:1019C000CE01DF91CF911F910F91FF90EF9008957D
:1019D000FD82EC82B801888199810E945025F0CF68
:1019E000FC011182108213821282158214820C94DF
:1019F000CB0CEF92FF920F931F93CF93DF93EC01E9
:101A00007B018A01BA010E94470C81110BC0CE01F3
:101A10000E942B0CCE01DF91CF911F910F91FF906F
:101A2000EF9008951D830C83B701888199810E94EE
:101A3000F530F0CFFB0101900020E9F73197AF01BD
:101A4000461B570B0C94F90C0F931F93CF93DF9306
:101A5000CDB7DEB762970FB6F894DEBF0FBECDBF2D
:101A60008C01CB01F801118210821382128215823F
:101A700014824AE0BE016F5F7F4F0E946025BE0165
:101A80006F5F7F4FC8010E941A0D62960FB6F894DF
:101A9000DEBF0FBECDBFDF91CF911F910F91089593
:101AA000CF93DF93EC01FB018617970749F0608124
:101AB00071816115710541F0448155810E94F90CD5
:101AC000CE01DF91CF9108950E942B0CF9CFFC013C
:101AD0001182108213821282158214820C94500D8E
:101AE000FC01118210821382128215821482FB0182
:101AF00001900020E9F73197AF01461B570B0C947A
:101B0000F90CAF92BF92CF92DF92EF92FF920F93B8
:101B10001F93CF93DF936C015B017A018901241736
:101B2000350720F48F2D7901042F182F60E572E01E
:101B3000C6010E94700DD5011496CD91DC91EC1672
:101B4000FD06E0F40C171D0708F4E801D501ED913E
:101B5000FC911197EC0FFD1F108110826D917C910B
:101B60006E0D7F1DC60161157105A1F00E941A0D51
:101B7000F50180819181C80FD91F1883C601DF91BB
:101B8000CF911F910F91FF90EF90DF90CF90BF907A
:101B9000AF9008950E942B0CEBCF0F931F93CF9320
:101BA000DF93CDB7DEB72C970FB6F894DEBF0FBE2C
:101BB000CDBFFC01248135811216130664F48C011B
:101BC000253131059CF40E94500364E170E080E00F
:101BD00090E00E9478052C960FB6F894DEBF0FBEF9
:101BE000CDBFDF91CF911F910F9108952FE030E08D
:101BF00050E040E0BC01CE0107960E94810DCE016D
:101C000007960E94470369E170E080E090E00E943F
:101C10007805F801248135814FE050E0B801CE010C
:101C200001960E94810DBE016F5F7F4FCE01079626
:101C30000E94F20BCE0101960E943D0CCE01079648
:101C40000E94500364E170E080E090E00E9478051B
:101C500060E572E0CE0107960E941A0DCE0107964C
:101C60000E943D0CB8CFEF92FF920F931F93CF933A
:101C7000DF93CDB7DEB7A1970FB6F894DEBF0FBEE6
:101C8000CDBF7C01CB01BA01F70111821082138212
:101C900012821582148242E0420F8E010F5F1F4FA5
:101CA0000E940725009789F0BC01C7010E941A0D08
:101CB000A1960FB6F894DEBF0FBECDBFDF91CF91D6
:101CC0001F910F91FF90EF900895C7010E942B0C78
:101CD000EFCF8F929F92AF92BF92EF92FF920F93AE
:101CE0001F93CF93DF93CDB7DEB72C970FB6F89441
:101CF000DEBF0FBECDBF64E670E080E090E00E94E2
:101D0000780580910B0290910C020B9731F5809130
:101D10005905882309F0F89482E10E94AB058C01F3
:101D200080915905882309F078940115110509F46B
:101D3000BDC080E090ECA9E7B4EC80934C05909393
:101D40004D05A0934E05B0934F0580935005909399
:101D50005105A0935205B093530580910B029091C9
:101D60000C02469731F580915905882309F0F894C3
:101D700081E00E94AB058C0180915905882309F010
:101D800078940115110509F4F2C080E090ECA9E700
:101D9000B4EC80934C0590934D05A0934E05B09301
:101DA0004F058093500590935105A0935205B09331
:101DB000530564E670E080E090E00E947805012B16
:101DC00009F063C040915005509151056091520552
:101DD0007091530521E0CE0107960E94330E61E514
:101DE00072E0CE0101960E94700DBE01695F7F4FC7
:101DF000CE0101960E94B10C64E572E00E949B0C3A
:101E0000BC0182E095E00E94500DCE0101960E9437
:101E10003D0C40914C0550914D0560914E057091DF
:101E20004F0521E0CE0101960E94330EBE016F5F87
:101E30007F4FCE0107960E94F20BCE0101960E94C1
:101E40003D0C68E572E0CE0101960E94700DBE0166
:101E5000695F7F4FCE0101960E94B10C6BE572E085
:101E60000E949B0CBC0182E095E00E94C40CCE0154
:101E700001960E943D0C64E670E080E090E00E94D4
:101E80007805CE0107960E943D0C2C960FB6F8946B
:101E9000DEBF0FBECDBFDF91CF911F910F91FF909D
:101EA000EF90BF90AF909F908F9008951091540540
:101EB000E09055056E2D70E090E080E00E94B22920
:101EC0002DEC3CEC4CEC5DE30E94112A4B015C01D3
:101ED000612F70E090E080E00E94B2299B01AC018C
:101EE000C501B4010E944C2B60934C0570934D05C5
:101EF00080934E0590934F0500915605F09057053D
:101F0000602F6F7770E090E080E00E94B2294B0173
:101F10005C016F2D70E090E080E00E94B2292DEC12
:101F20003CEC4CEC5DE30E94112A9B01AC01C50125
:101F3000B4010E944C2B07FD18C0609350057093AC
:101F4000510580935205909353051E0D100F1F0DE0
:101F500081E090E020915805121302C090E080E0EB
:101F600000271127081B190BF8CE9058E6CF1091C7
:101F700055050091540560915405709155057627DB
:101F80006727762790E080E00E94B0292DEC3CEC9A
:101F90004CEC5DE30E94112A60934C0570934D0553
:101FA00080934E0590934F05E0905705F0905605AD
:101FB0006F2D6F77762F6E2D90E080E00E94B02914
:101FC0002DEC3CEC4CEC5DE30E94112AF7FC18C0B0
:101FD000609350057093510580935205909353057B
:101FE000100F1E0D1F0D81E090E020915805121377
:101FF00002C090E080E000271127081B190BD9CE02
:102000009058E6CF0F931F93CF93DF938C01EB0192
:1020100088E2FB0111928A95E9F74BE050E06DE50B
:1020200072E0CE010E940A311B8681E090E0A0E0C0
:10203000B0E08C879D87AE87BF87F8018589968938
:10204000A789B08D888B998BAA8BBB8B82E090E09F
:10205000A0E0B0E08C8B9D8BAE8BBF8B1CA21DA231
:102060001EA21FA280E090E0A8E4B4E4888F998FBC
:10207000AA8FBB8F80E090E0A8E4B4EC8C8F9D8F9A
:10208000AE8FBF8F8DEC9CECACE4BEE388A399A32C
:10209000AAA3BBA3DF91CF911F910F910895AF9297
:1020A000BF92CF92DF92EF92FF920F931F93CF9345
:1020B000DF938C01EB0184E2FB0111928A95E9F731
:1020C0008EE10E940D0363E086E894E00E942709F8
:1020D0000E94340766E08EE10E941B08109298036C
:1020E000809397038630F0F30E94FA02A82E0E9494
:1020F000FA02B82E0E94FA02E82E0E94FA02F82E86
:102100000E94FA02C82E0E94FA02D82E60E07A2DB0
:102110006B29072E000C880B990B0E94B229F8013D
:10212000658376838783908760E07C2D6D29072EF9
:10213000000C880B990B0E94B229F8016187728705
:102140008387948760E07E2D6F29072E000C880B13
:10215000990B0E94B229F801658776878787908B53
:10216000118A128A138A148A84E290E0A0E0B0E017
:1021700088839983AA83BB8385899689A789B08D33
:102180008C839D83AE83BF8382E090E0A0E0B0E0CB
:1021900088879987AA87BB87188A198A1A8A1B8A0F
:1021A000C0900402D0900502E0900602F090070271
:1021B000A701960165817681878190850E942A2CEE
:1021C00020E030E048EC52E40E94112A6C8B7D8BB9
:1021D0008E8B9F8BA7019601F8016185728583859F
:1021E00094850E942A2C20E030E048EC52E40E94C2
:1021F000112A688F798F8A8F9B8F209100023091EE
:1022000001024091020250910302F8016585768532
:10221000878590890E942A2C20E030E048EC52E427
:102220000E94112A6C8F7D8F8E8F9F8F81E0DF91AE
:10223000CF911F910F91FF90EF90DF90CF90BF90C3
:10224000AF90089585ED8093BC008091C10390917B
:10225000C203A091C303B091C4030796A11DB11D91
:1022600023E0B695A795979587952A95D1F7209164
:10227000BC0024FD03C01092BF0308954091C10328
:102280005091C2036091C3037091C403452B462B48
:10229000472B69F30097A105B10541F025E32A9585
:1022A000F1F700000197A109B109E1CF8091C003C6
:1022B0000C9413074F925F926F927F928F929F922E
:1022C000AF92BF92CF92DF92EF92FF92CF93DF93C4
:1022D000CDB7DEB7CA54D1090FB6F894DEBF0FBE32
:1022E000CDBF60E572E0CE01C7960E94700D60E53B
:1022F00072E0CE01CD960E94700DBE016F5F7F4FE0
:1023000088E095E00E944F10CD88DE88EF88F88C39
:1023100020E030E040E251E4C701B6010E94112AFA
:102320002B013C01898D9A8DAB8DBC8D2B968CAF8A
:102330009DAFAEAFBFAF2B9720E030E040E251E45D
:10234000BC01CD010E94112A4B015C0120E030E06C
:1023500040E251E46D8D7E8D8F8D98A10E94112AEF
:1023600027966CAF7DAF8EAF9FAF2797C701B601A1
:1023700090582B962CAD3DAD4EAD5FAD2B970E9486
:10238000CB2B2BED3FE049EC5FE30E944C2B2091DF
:10239000A2043091A3044091A4045091A5040E948A
:1023A0004C2B6B017C0120E030E0A9010E94AB299D
:1023B00087FF0AC02BED3FE049EC50E4C701B601AE
:1023C0000E944C2B6B017C012BED3FE049EC50E46B
:1023D000C701B6010E94F92C181654F42BED3FE00A
:1023E00049EC50E4C701B6010E944B2B6B017C0104
:1023F00020E030E044E353E4C701B6010E94112A13
:102400002BED3FE049E450E40E942A2C6B017C0153
:1024100020E0BC01A601CE018B960E94330E65E63A
:1024200072E0CE0185960E94700DBE01655D7F4F02
:10243000CE0185960E94B10C6FE672E00E949B0C63
:10244000BC0182E095E00E94500DCE0185960E946D
:102450003D0CCE018B960E943D0C20E030E044EB19
:1024600052E4C701B6010E94AB2918160CF4BFC193
:1024700020E030E040E05FE3C701B6010E944C2B52
:10248000AB01BC0120E0CE018B960E94330E66E7C3
:1024900072E0CE0185960E94700DBE01655D7F4F92
:1024A000CE0185960E94B10CBC01CE01C7960E9458
:1024B000500DCE0185960E943D0CCE018B960E9458
:1024C0003D0C69E772E0CE01CD960E941A0D64E7DB
:1024D00072E0CE0185960E94700DBE01635C7F4F55
:1024E000CE0185960E94B10CBC01CE01C7960E9418
:1024F000C40CCE0185960E943D0C0E94A206C0909D
:102500001603D0901703E0901803F09019036C198C
:102510007D098E099F090E94B02920E030E04AE73A
:1025200054E40E942A2CAB01BC0123E0CE018B961F
:102530000E94330E69E872E0CE0185960E94700D0C
:10254000BE01655D7F4FCE0185960E94B10C60E8AB
:1025500072E00E949B0CBC018AEE94E00E94500D38
:10256000CE0185960E943D0CCE018B960E943D0CBB
:102570006AEE74E0CE0185960E94670DCE018596C5
:102580000E946B09CE0185960E943D0C62E075E0C9
:10259000CE0185960E94670DCE0185960E946B093B
:1025A000CE0185960E943D0CBE01695C7F4FCE0135
:1025B00085960E94670DCE0185960E94CD0DCE01B5
:1025C00085960E943D0C6AEE74E0CE0185960E94CD
:1025D000670D62E075E0CE0185960E94B10CBE01E8
:1025E000695C7F4F0E94B10CBC01CE01C7960E946E
:1025F000500DCE0185960E943D0C62EA73E0CE013B
:1026000085960E94F00CCE0185960E946B09CE0142
:1026100085960E943D0C60E572E082E095E00E94A4
:102620001A0D21E0B301A201CE0185960E94330E5E
:10263000BE016B5D7F4F82E095E00E94C40CCE012D
:1026400085960E943D0C21E027964CAD5DAD6EADA8
:102650007FAD2797CE01C1960E94330E21E0B501D0
:10266000A401CE018B960E94330E64E772E0CE0186
:1026700085960E94700DBE01655D7F4FCE018596E7
:102680000E94B10C64E772E00E949B0CBE016F5C7B
:102690007F4F0E94B10C63E872E00E949B0CBC016A
:1026A00082E095E00E94C40CCE0185960E943D0C0C
:1026B000CE018B960E943D0CCE01C1960E943D0C2E
:1026C00062E075E0CE0185960E94670DCE01859689
:1026D0000E946B09CE0185960E943D0CA3019201D8
:1026E000C301B2010E94112A6B017C01A501940172
:1026F000C501B4010E94112A9B01AC01C701B601BA
:102700000E944C2B6B017C0127962CAD3DAD4EAD4C
:102710005FAD2797CA01B9010E94112A9B01AC0144
:10272000C701B6010E944C2B0E945C2D6B017C01FD
:1027300067E872E082E095E00E941A0D21E0B7019F
:10274000A601CE0185960E94330EBE016B5D7F4FC0
:10275000CE018B960E94670D64E872E0CE018B96E5
:102760000E949B0CBC0182E095E00E94C40CCE014B
:102770008B960E943D0CCE0185960E943D0C62E036
:1027800075E0CE0185960E94670DCE0185960E9468
:10279000CD0DCE0185960E943D0C60E572E082E091
:1027A00095E00E941A0D65E070E080E090E00E94E4
:1027B0007805CE01CD960E943D0CCE01C7960E94B1
:1027C0003D0CC65BDF4F0FB6F894DEBF0FBECDBF2A
:1027D000DF91CF91FF90EF90DF90CF90BF90AF90BF
:1027E0009F908F907F906F905F904F90089520E022
:1027F00030E044E353E4C701B6010E94AB29181648
:1028000094F0A701960160E070E884E393E40E94ED
:102810004B2BAB01BC0120E0CE018B960E94330E06
:102820006BE772E036CE20E030E047E853E4C701C2
:10283000B6010E94AB29181694F120E030E044E381
:1028400053E4C701B6010E944B2B20E030E040E08A
:102850005FE30E944C2BAB01BC0120E0CE018B96C4
:102860000E94330E6BE772E0CE0185960E94700DD8
:10287000BE01655D7F4FCE0185960E94B10CBC0103
:10288000CE01C7960E94500DCE0185960E943D0C48
:10289000CE018B960E943D0C6EE772E014CEA7012C
:1028A000960160E070E084EB93E40E944B2B20E003
:1028B00030E040E05FE30E944C2B0E949C2CCE0154
:1028C0008B960E94240D66E772E0CECF4F925F9206
:1028D0006F927F928F929F92AF92BF92CF92DF9230
:1028E000EF92FF92CF93DF93CDB7DEB72C970FB661
:1028F000F894DEBF0FBECDBF0E94DA096B017C01E8
:102900000E94C2099C0150E040E0E1E2F5E08589C7
:102910009689281B390B41095109A389B4890E9462
:10292000072B4B015C018FE0B594A7949794879493
:102930008A95D1F765857685072E000C880B990B53
:102940002BE0660F771F881F991F2A95D1F72785DF
:102950003089032E000C440B550B280D391D4A1DE0
:102960005B1D0E94E82ACA01B901680D791D8A1D04
:102970009B1D685F7F4F8F4F9F4F34E095958795E4
:10298000779567953A95D1F70E94B2292B013C01C2
:1029900060919E0470919F048091A0049091A10485
:1029A0000E94B2294B015C010E94DA090E94B229FF
:1029B000A50194010E942A2C21E03EED42E45EE351
:1029C0000E94062D4B015C01C701B6010E94B2298D
:1029D00020E030E048EC52E40E942A2CAB01BC011C
:1029E00022E0CE0101960E94330EBE016F5F7F4F41
:1029F0008AEE94E00E94F20BCE0101960E943D0CFB
:102A000043E050E06DE073E08AEE94E00E946F0CCA
:102A10006AEE74E080EF94E00E94500D6CEE72E07C
:102A2000CE0101960E94700D6AEE74E0CE0101960F
:102A30000E94B10CBC018AEE94E00E94500DCE01C0
:102A400001960E943D0C66E773E082E095E00E94EB
:102A5000CB0C20E030E040E251E4C301B2010E941F
:102A60002A2CAB01BC0121E0CE0101960E94330E5D
:102A7000BE016F5F7F4F82E095E00E94C40CCE01E3
:102A800001960E943D0C45E050E06BE872E082E068
:102A900095E00E946F0CA501940160E070E080E871
:102AA0009FE30E944B2B20E03AE24DE257E40E9464
:102AB000112AAB01BC0121E0CE0101960E94330E28
:102AC000BE016F5F7F4FCE0107960E94670D61E9DF
:102AD00072E0CE0107960E949B0CBC0182E095E05B
:102AE0000E94C40CCE0107960E943D0CCE010196B7
:102AF0000E943D0C6AEE74E0CE0101960E94670DC3
:102B000064E772E0CE0101960E949B0C62E075E0E2
:102B10000E94B10CBC0182E095E00E94500DCE01F4
:102B200001960E943D0C65E070E080E090E00E941C
:102B300078052C960FB6F894DEBF0FBECDBFDF919F
:102B4000CF91FF90EF90DF90CF90BF90AF909F908C
:102B50008F907F906F905F904F9008952F923F924B
:102B60004F925F926F927F928F929F92AF92BF929D
:102B7000CF92DF92EF92FF920F931F93CF93DF9349
:102B8000CDB7DEB7CC55D1090FB6F894DEBF0FBE76
:102B9000CDBF29966CAF7DAF8EAF9FAF299725969D
:102BA0002CAF3DAF4EAF5FAF2597683E73408105B8
:102BB000910554F088E290E0A0E0B0E029968CAF57
:102BC0009DAFAEAFBFAF299725962CAD3DAD4EADB5
:102BD0005FAD25972115314E454F554054F020E00B
:102BE00031EE45EF55E025962CAF3DAF4EAF5FAFD0
:102BF000259780917203882351F081E090E0A0E056
:102C0000B0E025968CAF9DAFAEAFBFAF25970E94C9
:102C1000A20669966CAF7DAF8EAF9FAF69970E9499
:102C2000A2062D966CAF7DAF8EAF9FAF2D976996A4
:102C30006CAD7DAD8EAD9FAD699728EE33E040E081
:102C400050E00E94E82A6D962CAF3DAF4EAF5FAFCB
:102C50006D97772473941E0197E0290E311C2D96F1
:102C60006CAD7DAD8EAD9FAD2D9769962CAD3DAD14
:102C70004EAD5FAD6997621B730B840B950B259668
:102C80002CAD3DAD4EAD5FAD259762177307840740
:102C900095070CF0FEC20E94B22920E030E04AE71E
:102CA00054E40E942A2CAB01BC0123E0CE01019622
:102CB0000E94330EBE016F5F7F4F80EF94E00E9451
:102CC000F20BCE0101960E943D0C25968CAD9DAD78
:102CD000AEADBFAD25970A97A105B10524F518AA99
:102CE0001FA61AAA19AA1CAA1BAA2AE0AE014F5FA6
:102CF0005F4F6D966CAD7DAD8EAD9FAD6D970E94B3
:102D00006B25BE016F5F7F4FCE018F960E941A0D1B
:102D1000BE01615D7F4F80EF94E00E94F20BCE0117
:102D20008F960E943D0C80917203882361F160E5CB
:102D300072E080EF94E00E941A0D83E50E940D037B
:102D400062E386E894E00E9427090E94340783E545
:102D50000E940D0366E070E083E590E00E9479092F
:102D600008E315E0C801885395400F5F1F4F30916D
:102D7000970320919803321701F10E94FA02D801BB
:102D80001D968C93EFCF69E872E0CE0101960E9408
:102D9000700D60EF74E0CE0101960E94B10C60E806
:102DA00072E00E949B0CBC0180EF94E00E94500DE9
:102DB000CE0101960E943D0CC0CF069729F01092DB
:102DC0003805B1E0B09339050E943407809146057B
:102DD000909147059A838983809148059091490590
:102DE0009C838B8380914A0590914B059E838D83B4
:102DF0008E010F5F1F4F9AE3892E95E0992E2E01C9
:102E0000E3E24E0E511C5201D8016D917D918D016E
:102E1000F401C190D190E190F1904F01072E000C88
:102E2000880B990B0E94B229A70196010E94112AD2
:102E3000D5016D937D938D939D935D0102151305CF
:102E400019F760E572E082E095E00E941A0D8201B8
:102E5000045F1F4FC12CD12C7601F201819091901B
:102E6000A190B1902F01A5019401C501B4010E9468
:102E7000112A9B01AC01C701B6010E944C2B6B01CA
:102E80007C0123E0B501A401CE0101960E94330E1E
:102E9000BE016F5F7F4FCE018F960E94670D64E782
:102EA00072E0CE018F960E949B0CBC0182E095E0FF
:102EB0000E94C40CCE018F960E943D0CCE0101965B
:102EC0000E943D0C4016510641F6C701B6010E9412
:102ED0005C2D6B017C012DEC3CEC4CE45FE30E942B
:102EE000F92C18160CF080C12AE939E949E95FE3A9
:102EF000C701B6010E94AB2987FF76C1772009F48C
:102F000073C18BA49CA4ADA4BEA44BA05CA06DA077
:102F10007EA0CFA0D8A4E9A4FAA420E030E0A901C3
:102F2000C501B4010E94AB29882309F44AC1A30159
:102F30009201C301B2010E94112A61966CAF7DAF6C
:102F40008EAF9FAF6197A7019601C701B6010E949E
:102F5000112A9B01AC0161966CAD7DAD8EAD9FAD2C
:102F600061970E944C2B0E945C2DA50194010E9448
:102F7000CB2B20EE3EE245E652E40E94112A6196F8
:102F80006CAF7DAF8EAF9FAF619720E030E0A901BD
:102F9000C701B6010E94AB29882309F417C1A30118
:102FA0009201C301B2010E94112A65966CAF7DAFF8
:102FB0008EAF9FAF6597A5019401C501B4010E9432
:102FC000112A9B01AC0165966CAD7DAD8EAD9FADB8
:102FD00065970E944C2B0E945C2DA70196010E94D0
:102FE000CB2B20EE3EE245E652E40E94112A659684
:102FF0006CAF7DAF8EAF9FAF659720E030E0A90149
:10300000C301B2010E94AB29882309F4E4C0A501E1
:103010009401C501B4010E94112A4B015C01A70172
:103020009601C701B6010E94112A9B01AC01C5019E
:10303000B4010E944C2B0E945C2DA30192010E94BE
:10304000CB2B6B017C0160EF74E0CE0101960E94F6
:10305000670D63E972E0CE0101960E949B0CBC01F2
:1030600082E095E00E94500DCE0101960E943D0C39
:1030700062E075E0CE0101960E94670DCE010196D7
:103080000E946B09CE0101960E943D0C21E06196E1
:103090004CAD5DAD6EAD7FAD6197CE01CB960E941C
:1030A000330E21E065964CAD5DAD6EAD7FAD65979D
:1030B000CE01C5960E94330E20EE3EE245E652E474
:1030C000C701B6010E94112AAB01BC0121E0CE016B
:1030D00001960E94330EBE016F5F7F4FCE018F9627
:1030E0000E94670D64E772E0CE018F960E949B0CF0
:1030F000BE016B5C7F4F0E94B10C64E772E00E94DE
:103100009B0CBE01655C7F4F0E94B10CBC0182E04C
:1031100095E00E94500DCE018F960E943D0CCE018D
:1031200001960E943D0CCE01C5960E943D0CCE0139
:10313000CB960E943D0C62E075E0CE0101960E94A4
:10314000670DCE0101960E94CD0DCE0101960E9421
:103150003D0C60E572E082E095E00E941A0D772454
:10316000739460E572E082E095E00E941A0D0E947F
:10317000A206DC01CB012D962CAD3DAD4EAD5FAD71
:103180002D97821B930BA40BB50B29962CAD3DAD4F
:103190004EAD5FAD299782179307A407B50744F496
:1031A000281B390B4A0B5B0BCA01B9010E94780539
:1031B0000E94A2062D966CAF7DAF8EAF9FAF2D976C
:1031C0004ECD6BED7FE089EC9FE3D3CE6BED7FE0DE
:1031D00089EC9FE306CF8BEDC82E8FE0D82E89ECCB
:1031E000E82E8FE3F82E2FCF69E673E0CE0101962B
:1031F0000E94F00CCE0101960E946B09CE0101964F
:103200000E943D0C62E075E0CE0101960E94670DC0
:10321000CE0101960E94CD0DCE0101960E943D0C7B
:1032200023E0B701A601CE018F960E94330E60EF16
:1032300074E0CE0101960E94670D6BEA72E0CE0148
:1032400001960E949B0CBE01615D7F4F0E94B10CF4
:103250006EEA72E00E949B0CBC0182E095E00E9445
:10326000500DCE0101960E943D0CCE018F960E941A
:103270003D0C62E075E0CE0101960E94670DCE0123
:1032800001960E94CD0DCE0101960E943D0C712C3D
:1032900068CFC45ADF4F0FB6F894DEBF0FBECDBF64
:1032A000DF91CF911F910F91FF90EF90DF90CF9022
:1032B000BF90AF909F908F907F906F905F904F9056
:1032C0003F902F9008954F925F926F927F928F92CE
:1032D0009F92AF92BF92CF92DF92EF92FF920F93A5
:1032E0001F93CF93DF9300D000D0CDB7DEB78C0112
:1032F00060E572E082E095E00E941A0DC801059633
:10330000059740F00C3E2FEF120724F010936A034C
:10331000009369030130110509F4E3C00CF061C0AA
:103320000B3F3FEF1307C4F4093F4FEF140744F579
:10333000083F5FEF15070CF0B6C0013F8FEF18078D
:10334000FCF4083E1F4F09F4AAC164E973E082E06F
:1033500095E00E94CB0C14C00D3FFFEF1F0709F44E
:10336000B4C05CF40B3F3FEF130709F49FC00C3F60
:103370001F4F59F71092720303C00F3F1F4F2CF3DA
:103380008091060590910705892B71F062E075E048
:10339000CE0101960E94670DCE0101960E94CD0DCF
:1033A000CE0101960E943D0C64E670E080E090E062
:1033B0000E94780526960FB6F894DEBF0FBECDBFEB
:1033C000DF91CF911F910F91FF90EF90DF90CF9001
:1033D000BF90AF909F908F907F906F905F904F9035
:1033E00008950930110544F5073011054CF60430F5
:1033F000110509F481C04CF40230110509F474C0C0
:103400000330110509F4BCCFA0CF0530110509F434
:1034100093C00630110509F098CF809108028823E7
:1034200009F4AECF80917203882309F48FC082E043
:1034300090E00E945A11A4CF0331110549F064F5C0
:103440000930110509F4F2C00C30110509F07DCFE7
:1034500080910802882309F493CF0D31110509F0FA
:1034600022C10E94661462E075E0CE0101960E94BE
:10347000670DCE0101960E94CD0DCE0101960E94EE
:103480003D0C64EF71E080E090E00E9478050C3024
:10349000110509F475CFCFC00D311105C9F20138FE
:1034A0001105B1F252CF0E94A2066ACF8091720339
:1034B000882321F082E095E00E94500368EC70E0E0
:1034C00080E090E00E9478055BCF81E080937203FA
:1034D0008091690390916A0390936D0380936C03CC
:1034E0004FCF0E94690E4CCF80910802882309F4C7
:1034F00047CF0E94661444CF81E0809315020E945A
:103500002E068C0169E773E082E095E00E94CB0C07
:1035100060E074E0601B710BCE0101960E94240DE7
:10352000BE016F5F7F4F82E095E00E94C40CCE0128
:1035300001960E943D0C24CF69E873E082E095E09B
:103540000E94CB0C0E942E06BC01E6CF20E030E0AA
:103550004AE754E460910D0270910E0280910F02CF
:10356000909110020E94112A0E949C2C4B015C0138
:1035700020E030E04AE754E46091110270911202B9
:1035800080911302909114020E94112A0E949C2C97
:103590006B017C0189EEC81683E0D806E104F104D2
:1035A0002CF084E1C82ED12CE12CF12C0E94A20633
:1035B0006093160370931703809318039093190375
:1035C0000E94A2062B013C018091160390911703E3
:1035D000A0911803B0911903A3019201281B390B84
:1035E0004A0B5B0BDA01C90188159905AA05BB05D1
:1035F0000CF0C6CE83E090E00E945A110E94A20611
:10360000DC01CB0184199509A609B7098C159D0524
:10361000AE05BF05ACF6A7019601281B390B4A0B76
:103620005B0BCA01B9010E947805CACF80910802DC
:10363000882309F4A5CE80917203882359F021E0F4
:1036400030E040E050E06AE070E080E090E00E940E
:10365000AE1596CE20E030E04AE754E460910D02CA
:1036600070910E0280910F02909110020E94112A17
:103670000E949C2C6B017C0120E030E04AE754E47E
:1036800060911102709112028091130290911402C4
:103690000E94112A0E949C2CA7019601D8CFF0E02D
:1036A000E0E019956DCE64EF71E080E090E00E945B
:1036B00078050E94690E0331110509F4BCCFD1CE03
:1036C0001F920F920FB60F9211240BB60F922F93E9
:1036D0003F934F935F936F937F938F939F93AF939A
:1036E000BF93EF93FF9389EE93E00E94A903FF91AC
:1036F000EF91BF91AF919F918F917F916F915F916A
:103700004F913F912F910F900BBE0F900FBE0F90D6
:103710001F9018951F920F920FB60F9211240BB69F
:103720000F922F938F939F93EF93FF93E091F90361
:10373000F091FA038081E091FF03F091000482FD93
:103740001DC09081809102048F5F8F7320910304CC
:10375000821741F0E0910204F0E0E751FC4F958FB1
:1037600080930204FF91EF919F918F912F910F9081
:103770000BBE0F900FBE0F901F9018958081F2CF57
:103780001F920F920FB60F9211242F933F938F9396
:103790009F93AF93BF9380915F0390916003A0913B
:1037A0006103B091620330915E0323E0230F2D3754
:1037B00058F50196A11DB11D20935E0380935F0310
:1037C00090936003A0936103B093620380916303BD
:1037D00090916403A0916503B09166030196A11DC9
:1037E000B11D8093630390936403A0936503B0932A
:1037F0006603BF91AF919F918F913F912F910F9051
:103800000FBE0F901F90189526E8230F0296A11D5A
:10381000B11DD2CF1F920F920FB60F9211240BB68B
:103820000F922F933F934F935F936F937F938F9359
:103830009F93AF93BF93EF93FF938091B900887FDD
:10384000803609F44DC008F040C0883209F4A9C0A0
:1038500028F5803109F49DC0C8F4882309F4FBC021
:10386000883009F496C0FF91EF91BF91AF919F917D
:103870008F917F916F915F914F913F912F910F9019
:103880000BBE0F900FBE0F901F901895883109F452
:1038900088C0803241F78093BD0314C0803409F49E
:1038A0009DC040F48033B9F38833E9F68093BD03BB
:1038B00085ECB0C0803509F485C0883509F496C020
:1038C000883489F60E942211CECF883909F48CC041
:1038D00038F5883729F050F4883611F0803719F61A
:1038E00083E08093BF0310925D0357C0883809F4CA
:1038F0007BC0803919F0803809F0B5CF80915D0325
:10390000803208F071C0E0915D0381E08E0F8093FA
:103910005D038091BB00F0E0E35CFC4F80833DC021
:10392000803B39F0E0F4803A09F479C0883A09F034
:103930009ACF84E08093BF0310923C0310923B0324
:10394000E0917503F0917603199580913B03811105
:103950000FC081E080933B0310921B0309C0803CA1
:1039600009F4A6CF883C09F4A3CF883B09F07BCFAC
:10397000E0913C0381E08E0F80933C03F0E0E55E34
:10398000FC4F80818093BB0090913C0380913B036E
:1039900029C080919A038093BB0085EC8093BC0082
:1039A00062CF9091BC038091BB03981758F5E091CA
:1039B000BC0381E08E0F8093BC03F0E0E556FC4F22
:1039C0008081E9CFE091BC0381E08E0F8093BC033E
:1039D0008091BB00F0E0E556FC4F80839091BC03E2
:1039E0008091BB039817C8F285E8D8CFE091BC035B
:1039F00081E08E0F8093BC038091BB00F0E0E55620
:103A0000FC4F80838091BE0381115CCF81E0809365
:103A1000990384EA8093BC001092BF0324CF85EC05
:103A20008093BC001092BF0380915D03803230F41C
:103A3000E0915D03F0E0E35CFC4F108260915D0378
:103A400070E0E0917303F09174038DE393E01995B6
:103A500010925D0308CF1092BD0334CFCF93DF9354
:103A6000E9EEF3E01382128288EE93E0A0E0B0E08A
:103A700084839583A683B78320E232E03183208359
:103A800025EC30E03587248724EC30E03787268723
:103A900020EC30E0318B208B21EC30E0338B228B1B
:103AA00022EC30E0358B248B26EC30E0378B268BF4
:103AB000118E128E138E148EE6E8F4E013821282B9
:103AC00084839583A683B78382E392E09183808386
:103AD00010925905E8E3F5E0C1E0C083118283EC60
:103AE0009BEAA6E7BBE382839383A483B58388ED37
:103AF0009BE6A6E7BBE386839783A087B18782EF27
:103B000094EEA4E6BBE382879387A487B587E8E0B9
:103B1000F5E084E492E0918380838FEF9FEFDC01F6
:103B2000858B968BA78BB08F60E572E082E095E085
:103B30000E94700D60E572E08CEF94E00E94700DC1
:103B400060E572E086EF94E00E94700D60E572E03F
:103B500080EF94E00E94700D60E572E08AEE94E0E0
:103B60000E94700D61EB72E084EE94E00E94700D93
:103B700068EB72E08EED94E00E94700DE2E9F4E0F3
:103B800086E190E0918380838CE79CE8A1E0B0E03F
:103B900084879587A687B78781EA97E6A3E3BDEB7D
:103BA000808B918BA28BB38B86E696E6A6EABFE369
:103BB000848B958BA68BB78BC0A389E190E092A3F1
:103BC00081A3C3A380E090E4ACE1B5E484A395A312
:103BD000A6A3B7A310A611A612A613A6AEEBB4E037
:103BE00080E1ED0119928A95E9F714AE15AE16AE93
:103BF00017AE1092D2041092D3041092D4041092F3
:103C0000D5041092D6041092D7041092D8041092C2
:103C1000D9041092DA041092DB041092DC041092A2
:103C2000DD04DF91CF910895CF93DF93CDB7DEB759
:103C3000AE970FB6F894DEBF0FBECDBF789484B5B3
:103C4000826084BD84B5816084BD85B5826085BD98
:103C500085B5816085BD80916E00816080936E0026
:103C60001092810080918100826080938100809118
:103C700081008160809381008091800081608093C9
:103C800080008091B10084608093B1008091B00089
:103C900081608093B0008091910082608093910058
:103CA000809191008160809391008091900081606B
:103CB000809390008091A10082608093A100809108
:103CC000A10081608093A1008091A0008160809319
:103CD000A0008091210182608093210180912101C7
:103CE0008160809321018091200181608093200177
:103CF00080917A00846080937A0080917A0082605B
:103D000080937A0080917A00816080937A0080911C
:103D10007A00806880937A001092C10061E086E3A7
:103D20000E942205E091F903F091FA0382E080837A
:103D3000E091F503F091F6031082E091F703F09122
:103D4000F8038FEC808310920104E091FD03F09161
:103D5000FE0386E08083E091FB03F091FC03808109
:103D600080618083E091FB03F091FC038081886097
:103D70008083E091FB03F091FC0380818068808365
:103D8000E091FB03F091FC0380818F7D808361E0F3
:103D900088E30E94220560E088E30E94F40461E069
:103DA00086E30E94F40468EC70E080E090E00E94FA
:103DB000780584E690E090930A02809309020E94BD
:103DC000D22A8093670385E690E00E94D22A8093EE
:103DD00068030091670310916803B801012E000C7D
:103DE000880B990B0E94B2299B01AC010E94A02D67
:103DF000811106C00B5011090C30110508F48CC05C
:103E000084E690E00E949F0B68EC70E080E090E018
:103E10000E9478056EEE73E082E095E00E94CB0C84
:103E200062E075E0CE0101960E94670DCE01019619
:103E30000E94CD0DCE0101960E943D0C0E94FC0611
:103E400064E670E080E090E00E94780583E0809373
:103E500021050E94FC0680ED0E948009853509F449
:103E600086C062EE73E082E095E00E94CB0C109277
:103E7000080262E075E0CE0101960E94670DCE0156
:103E800001960E94CD0DCE0101960E943D0C772433
:103E9000739488EE882E83E0982EA12CB12CF12CFF
:103EA000E12C9AE2C92ED12C60E572E0CE01899610
:103EB0000E94700D10E089EE93E00E9493031816A3
:103EC00019060CF0FEC01111FCC089EE93E00E94AF
:103ED00071038A3009F046C110916B03112309F474
:103EE00056C18091FA049091FB04892B09F448C1D2
:103EF00061EC72E0CE0101960E94700DBE01675D1B
:103F00007F4FCE0101960E94B10C0E945003CE015A
:103F100001960E943D0C34C122E9E22E24E0F22EEB
:103F200004E610E0C8010E94D22AF70181937F01C4
:103F30000F5F1F4F003B1105A9F7809192049091EC
:103F4000930490930C0280930B0264E974E0CE0119
:103F500001960E94700DBE016F5F7F4F84EE94E06A
:103F60000E94F20BCE0101960E943D0C4DCF8AEAD1
:103F70000E949D0990932305809322058CEA0E945C
:103F80009D0990932505809324058EEA0E949D0942
:103F9000909327058093260580EB0E949D099093BE
:103FA00033058093320582EB0E949D09909335057D
:103FB0008093340584EB0E949D099093370580938C
:103FC000360586EB0E949D0990932905809328056C
:103FD00088EB0E949D0990932B0580932A058AEB1C
:103FE0000E949D0990932D0580932C058CEB0E94D7
:103FF0009D0990932F0580932E058EEB0E949D09BD
:10400000909331058093300564EF71E080E090E09B
:104010000E9478050E94FC0680E00E94560980E11B
:104020000E94560988E00E9456090E94FC068EE113
:104030000E940D0362E086E894E00E94270960E098
:1040400086E894E00E9427090E9434078EE10E94CE
:104050000D0361E086E894E00E94270960E286E8AB
:1040600094E00E9427090E94340780E290E0909338
:104070000C0580930B0580E090E8A9E8B4E48093F8
:10408000040290930502A0930602B093070280E019
:1040900090E0A5E7B4E48093000290930102A0931E
:1040A0000202B0930302BE016F5F7F4F88E095E08C
:1040B0000E94021064EF71E080E090E00E947805B9
:1040C000E6CE8DA59EA5892B51F089EE93E00E9446
:1040D000180464E170E080E090E00E947805BE0181
:1040E000675D7F4F86EF94E00E94F20BCE018996C8
:1040F0000E943D0C60E572E082E095E00E941A0D9E
:104100008091FA049091FB048130910509F076C00A
:1041100066EF74E0CE0101960E94670D8D819E814D
:10412000892B91F0E981FA81309771F08081823496
:1041300009F44BC074F58A3209F45DC08134F1F1A1
:1041400063ED72E08332E1F1BE016F5F7F4F86EF76
:1041500094E00E94500D6AE070E080E090E00E94E0
:1041600078053FC08D3009F4B7CE89831A8241E0CB
:1041700050E0BE016F5F7F4FCE0189960E946F0CA9
:104180006AE070E080E090E00E94780594CE11E053
:10419000F7CF813699F06CF48334B1F660ED72E0BC
:1041A00086EF94E00E941A0D709272038DEF9FEFDC
:1041B00016C0823651F0833689F3C6CF6AEC72E0BE
:1041C00086EF94E00E941A0D0CC06DEC72E086EF51
:1041D00094E00E941A0D109272038CEF9FEF0E94E0
:1041E0006319CE0101960E943D0C86EF94E00E9477
:1041F000CC0BCB012FC066ED72E0E2CF049778F5CF
:1042000069ED72E0CE0101960E94700DBE016F5FF4
:104210007F4F86EF94E00E94D70B182FCE010196B6
:104220000E943D0C1123D9F08091FA049091FB0477
:10423000029798F0E091F604F091F704309769F056
:10424000818180330CF4845E9601281B310987FD3F
:104250003395C9010E94631934C080E0F4CF66EF42
:1042600074E08CEF94E00E94500D0091FC041091DA
:10427000FD040115110571F0F80181918F0188236A
:1042800049F0082E000C990B0E94E430F801319798
:104290008083F2CF61E774E0CE0101960E94F00CBA
:1042A000BE016F5F7F4F8CEF94E00E94D70B182FF9
:1042B000CE0101960E943D0C112309F448C0F7017C
:1042C000199580917203882309F43EC00E94A206CA
:1042D000A50194010E941A2BCA01B9010E94B029BC
:1042E00020916E0330916F034091700350917103E0
:1042F0000E944B2B20911102309112024091130227
:10430000509114020E94F92C1816F4F40E94A2068F
:10431000A50194010E941A2BCA01B9010E94B0297B
:1043200060936E0370936F03809370039093710397
:1043300080916C0390916D030E9463196AE070E0B4
:1043400080E090E00E9478050E943804ADCD69E6D7
:1043500074E0CE0101960E94F00CBE016F5F7F4FAA
:104360008CEF94E00E94D70B182FCE0101960E948B
:104370003D0C112399F16BED72E0CE0101960E9484
:10438000700D6EED74E0CE0101960E94B10CBC017F
:1043900082E095E00E94500DCE0101960E943D0CF6
:1043A00065EE72E0CE0101960E94700D62E075E04C
:1043B000CE0101960E94B10CBC01CE0189960E94EB
:1043C000670DCE0189960E94CD0DCE0189960E947F
:1043D0003D0CCE0101960E943D0C73CF62E674E065
:1043E000CE0101960E94F00CBE016F5F7F4F8CEFF3
:1043F00094E00E94D70B182FCE0101960E943D0C2D
:10440000112369F064E574E082E095E00E94CB0C32
:1044100064EE74E082E095E00E94C40CC1CF6DE4CC
:1044200074E0CE0101960E94F00CBE016F5F7F4FD9
:104430008CEF94E00E94D70B182FCE0101960E94BA
:104440003D0C112309F127E030E046E050E066EF33
:1044500074E0CE0101960E94810DBE016F5F7F4F17
:1044600080EF94E00E94F20BCE0101960E943D0C79
:1044700080EF94E00E94CC0B672B19F410926B0331
:1044800020CF70926B031DCF66E474E0CE010196DD
:104490000E94F00CBE016F5F7F4F8CEF94E00E9492
:1044A000D70B182FCE0101960E943D0C112309F461
:1044B0007EC02091FA043091FB042730310508F4C6
:1044C00000CF46E050E066EF74E0CE0101960E9416
:1044D000810DBE016F5F7F4F80EF94E00E94F20B71
:1044E000CE0101960E943D0C8091F0049091F10460
:1044F000009709F458C00E9425256093110270931B
:10450000120280931302909314026BE374E082E032
:1045100095E00E94CB0C40911102509112026091E3
:1045200013027091140222E0CE0101960E94330E14
:10453000BE016F5F7F4FCE0189960E94670D67EEC7
:1045400072E0CE0189960E949B0CBC0182E095E04E
:104550000E94C40CCE0189960E943D0CCE010196AA
:104560000E943D0C62E075E0CE0101960E94670D4D
:10457000CE0101960E94CD0DCE0101960E943D0C08
:104580000E94A206A50194010E941A2BCA01B9013A
:104590000E94B02960936E0370936F038093700341
:1045A000909371038ECE60E070E0CB01A6CF64E300
:1045B00074E0CE0101960E94F00CBE016F5F7F4F48
:1045C0008CEF94E00E94D70B182FCE0101960E9429
:1045D0003D0C112309F46CC02091FA043091FB04C6
:1045E0002730310508F46DCE46E050E066EF74E008
:1045F000CE0101960E94810DBE016F5F7F4F80EF5B
:1046000094E00E94F20BCE0101960E943D0C809135
:10461000F0049091F104009709F446C00E9425250A
:1046200060930D0270930E0280930F02909310021C
:1046300069E274E082E095E00E94CB0C40910D02AB
:1046400050910E0260910F027091100221E0CE0194
:1046500001960E94330EBE016F5F7F4FCE01899697
:104660000E94670D67EE72E0CE0189960E949B0C56
:10467000BC0182E095E00E94C40CCE0189960E94A4
:104680003D0CCE0101960E943D0C62E075E0CE012A
:1046900001960E94670DCE0101960E94CD0DCE01BC
:1046A00001960E943D0C0DCE60E070E0CB01B8CFCA
:1046B00064E274E0CE0101960E94F00CBE016F5FCF
:1046C0007F4F8CEF94E00E94D70B182FCE010196FC
:1046D0000E943D0C112341F126E030E044E050E01F
:1046E00066EF74E0CE0101960E94810DBE016F5FFE
:1046F0007F4F80EF94E00E94F20BCE0101960E9462
:104700003D0C80EF94E00E94CC0B70939304609377
:10471000920470930C0260930B02809109029091B5
:104720000A020E949F0BCDCD60E274E0CE0101969B
:104730000E94F00CBE016F5F7F4F8CEF94E00E94EF
:10474000D70B182FCE0101960E943D0C112309F4BE
:1047500051C02091FA043091FB0443E050E066EF31
:1047600074E0CE0101960E94810DBE016F5F7F4F04
:1047700080EF94E00E94F20BCE0101960E943D0C66
:1047800060EF74E0CE0101960E94670D19A61AA68B
:1047900041E050E0BE01675D7F4FCE0101960E946F
:1047A0006F0C811104C0CE0101960E942B0CBE013A
:1047B0006F5F7F4F84EE94E00E94500DCE01019612
:1047C0000E943D0C0091E8041091E90401151105C7
:1047D00009F4A3CF015011096091E4047091E5043C
:1047E000A80184E994E00E940A31F801EC56FB4FDD
:1047F000108293CF6DE174E0CE0101960E94F00C1F
:10480000BE016F5F7F4F8CEF94E00E94D70B182F93
:10481000CE0101960E943D0C112309F48CC0209119
:10482000FA043091FB042031310508F04ACD42E012
:1048300050E066EF74E0CE0101960E94810DBE014A
:104840006F5F7F4F80EF94E00E94F20BCE010196E4
:104850000E943D0C8091F0049091F104009799F131
:104860000E94252520E030E048EC52E40E94112A05
:104870000E949C2C60939E0470939F048093A004DC
:104880009093A1048B019C0100591F4521403109DF
:1048900001341C4921053105D0F069EE72E0CE01EA
:1048A00001960E94700D60EF74E0CE0101960E94A7
:1048B000B10C6FEE72E00E949B0CBC0182E095E0AF
:1048C0000E94500D86CD60E070E0CB01CBCF0E94FE
:1048D000B22920E030E048EC52E40E942A2CAB01DF
:1048E000BC0122E0CE0101960E94330EBE016F5F33
:1048F0007F4F82E095E00E94F20BCE0101960E946C
:104900003D0C6FEF72E0CE0101960E94700D62E0E7
:1049100075E0CE0101960E94B10C6CE073E00E943C
:104920009B0CBC0182E095E00E94500DCE010196E7
:104930000E943D0CF2CE61E173E0CE0101960E942F
:10494000700DBE016F5F7F4F8CEF94E00E94D70B1C
:10495000182FCE0101960E943D0C112339F06EE014
:1049600074E082E095E00E94CB0C8FCE6AE074E0A8
:10497000CE0101960E94F00CBE016F5F7F4F8CEF5D
:1049800094E00E94D70B182FCE0101960E943D0C97
:10499000112309F496CC2091FA043091FB0443E0F2
:1049A00050E066EF74E0CE0101960E94810DBE01D9
:1049B0006F5F7F4F80EF94E00E94F20BCE01019673
:1049C0000E943D0C80EF94E00E94CC0B70936A0330
:1049D000609369030ECC8EED94E00E943D0C84EE52
:1049E00094E00E943D0C8AEE94E00E943D0C80EF22
:1049F00094E00E943D0C86EF94E00E943D0C8CEF09
:104A000094E00E943D0C82E095E00C943D0CEF9206
:104A10000F931F93CF93DF93E80134E047FD34E118
:104A2000042E000C550B57FF03C0519541955109B9
:104A3000E32E022F242FAE010E94CB25CE01DF9161
:104A4000CF911F910F91EF900895662777270C94CF
:104A500044271F93FC0199278827BC01E8941191F2
:104A60001032E9F3193010F01E30C8F31B3251F048
:104A70001D3249F4689406C00E947A25610F711DA9
:104A8000811D911D119110531A30B0F33EF4909591
:104A90008095709561957F4F8F4F9F4F1F9108951F
:104AA000FB01DC0105900D920020E1F70895FC0167
:104AB00005900020E9F7809590958E0F9F1F08952F
:104AC000BB274A3031F4992322F4BDE290958195B9
:104AD0009F4F0C94B225BB272A3051F4992342F4FE
:104AE000BDE290958095709561957F4F8F4F9F4F58
:104AF0000C949025592F482F372F262F660F771F9C
:104B0000881F991F660F771F881F991F620F731FD9
:104B1000841F951F660F771F881F991F0895BB2755
:104B2000FA01A62F6217710581059105330B30FB41
:104B300066F0AA27660F771F881F991FAA1FA21762
:104B400010F0A21B63953850A9F7A05DAA3308F0B6
:104B5000A95DA19336F7B111B1931082CA010C94EB
:104B60009B29BB27FB015527AA27880F991FAA1F3E
:104B7000A41710F0A41B83955051B9F7A05DAA3378
:104B800008F0A95DA193009779F7B111B193119243
:104B9000CB010C949B298F929F92AF92BF92CF92A0
:104BA000DF92EF92FF920F931F93CF93DF9300D08A
:104BB00000D000D0CDB7DEB76A01F22EB02E102F94
:104BC000FBE3AF2EA01608F41BE31F5F012F27E0C5
:104BD000AE014F5F5F4F0E94A228BC018981982FD0
:104BE0009970913009F44EC09BE2E1FC04C09E2D07
:104BF0009170E0FC49C05E2D5071E82FE87083FF92
:104C000055C084E0911101C083E0EF2DE81B8F15A2
:104C100008F0E0E0D6018E2F20E25523C9F1992358
:104C200029F0D6019C93C60101966C0196012D5F77
:104C30003F4FE2FE33C08EE4D6018C9391E411968F
:104C40009C93119712968C93D9018E2F90E281112B
:104C50002AC0E20FF32FF11D10828EEF9FEF2996ED
:104C60000FB6F894DEBF0FBECDBFDF91CF911F917D
:104C70000F91FF90EF90DF90CF90BF90AF909F90FB
:104C80008F9008959DE2B7CF90E2B5CF2D938150DC
:104C90008111FCCFCE0ED11CE0E0C1CF8EE6D60153
:104CA0008C9391E6CCCF9D938150D1CF482F447007
:104CB00082FF3DC084E0911101C083E08F1510F4A4
:104CC000EF2DE81BD6018E2F20E2552309F1992301
:104CD00029F0D6019C93C60101966C0196012D5FC7
:104CE0003F4FE2FE1BC089E4D6018C938EE41196FF
:104CF0008C93119786E412968C93D9018E2F90E2B3
:104D0000882309F4A6CF9D938150FACF2D9381502B
:104D10008111FCCFCE0ED11CE0E0D9CF89E6D601BF
:104D20008C938EE611968C93119786E6E4CF9B01C7
:104D300077FF02C030E020E0A1E0B0E0911102C0B6
:104D4000B0E0A0E0F9013196AE0FBF1F8B2C912C83
:104D5000BB2009F461C05401EFEFAE1ABE0AAA0DE0
:104D6000BB1DFA161B0619F014F04F2D4A1B5111EA
:104D700088C0E3FC59C07601A42FB0E2A1114FC056
:104D8000C40ED11C992309F45BC040E0D6011196F2
:104D9000F60190836D01552309F448C0012F060FD9
:104DA0009A81582F507184FF03C0913309F4015048
:104DB00010160CF047C0093008F008E0EEE2FE2EB5
:104DC0005B01A01AB10885019194819491082F3F4D
:104DD000320729F4D601FC92F60131966F01621771
:104DE000730794F1021713077CF5DB01A21BB30BC9
:104DF000AA24A394B12CAC0EBD1EAA0DBB1D119606
:104E00008C9121503109D601119628153905F4F0FD
:104E1000F60180836D01DBCFB12CA12CA0CFF7016F
:104E2000B1937F01A150AACF9111B0CFD601942F99
:104E300050E302C05D9391509111FCCFC40ED11C80
:104E400040E0ACCF01E0BACF80E3DBCF621773075D
:104E500031F4963388F4953311F4552369F0F60153
:104E60008083FD01842F90E2811108C0A40FB11D41
:104E70001C9290E080E0F3CE81E3F1CF91938150DA
:104E8000F3CF911183CF8ACF8F929F92AF92BF922F
:104E9000CF92DF92EF92FF920F931F93CF93DF9306
:104EA0005C017B016115710519F0DB018D939C9309
:104EB00085010F5F1F4FF501D0818D2F90E00E947B
:104EC0007A296C01892BB9F5DD32B9F50F5F1F4FD7
:104ED000D5011196DC91C1E05801F1E0AF1AB1089B
:104EE00043E050E06CE372E0C5010E948329892B06
:104EF00069F5680182E0C80ED11C45E050E067E327
:104F000072E0C6010E948329892B21F4680197E091
:104F1000C90ED11CE114F10419F0D701CD92DC9235
:104F200060E070E080E89FEFC111FFC060E070E0DA
:104F300080E89FE7FAC05801BBCFDB3229F4850136
:104F40000E5F1F4FF501D181C0E0C6CF43E050E0B6
:104F500064E372E0C5010E948329892BE9F0F8011E
:104F600010E000E020E030E0A9015F01B0ED8B2E01
:104F70008D0E89E08815C8F19C2E689491F88C2FCD
:104F80008870C2FF16C0811102C00F5F1F4F31969B
:104F9000D501DC91C92DE9CFE114F10429F00E5FB0
:104FA0001F4FF7011183008360E070E080EC9FE702
:104FB000BCC0882311F001501109A5E0B0E00E94A7
:104FC000072B9B01AC01220F331F441F551F280DD7
:104FD000311D411D511D283999E93907490799E1CA
:104FE0005907A8F2C6609C2ED2CFAEEF8A1206C037
:104FF000C3FD3CC09C2E689493F8C9CFDF7DD534A7
:10500000A9F580818D3239F4C061DF01129681816A
:1050100062E070E006C0DF018B32C1F3119661E0FF
:1050200070E080535D01A61AB70A8A30F8F4E0E810
:10503000CE16ECE0DE065CF4B601660F771F660F55
:10504000771FC60ED71ECC0CDD1CC80ED11C5D010F
:10505000FFEFAF1ABF0A8C9180538A30A8F1C4FFCA
:1050600003C0D194C194D1080C0D1D1DC1FF09C00E
:10507000E114F10431F081E0A81AB108D701AD9232
:10508000BC92CA01B9010E94B029C370C33009F4AF
:1050900090584B015C0120E030E0A9010E94AB294F
:1050A000882309F440C0CBE6D2E017FF05C0119574
:1050B00001951109C3E5D2E06E01B8E1CB1AD10820
:1050C00080E2E82EF12C0FC0D501B1CFFE01259171
:1050D0003591459154910E191F09C501B4010E94E3
:1050E000112A4B015C01D501C4010E151F0574F78F
:1050F0002497F594E794CC16DD06A9F78A2F880F3C
:105100008B2F881F8F3F49F020E030E0A901C501B7
:10511000B4010E94AB29811106C082E290E0909315
:105120005B0580935A05C501B401DF91CF911F91B2
:105130000F91FF90EF90DF90CF90BF90AF909F9036
:105140008F900895283008F027E03327DA01990F6F
:10515000311D87FD916000966105710539F432605B
:105160002E5F3D9330E32A95E1F708959F3F30F09D
:1051700080387105610509F03C5F3C5F3D939130DB
:1051800008F08068911DDF93CF931F930F93FF92D8
:10519000EF92192F987F9695E92F96959695E90F9E
:1051A000FF27E753FD4F99273327EE24FF24A7015C
:1051B000E70105900894079428F4360FE71EF81EBF
:1051C000491F511D660F771F881F991F0694A1F76D
:1051D0000590079428F4E70EF81E491F561FC11DBD
:1051E000770F881F991F661F0694A1F705900794F3
:1051F00028F4F80E491F561FC71FD11D880F991F8D
:10520000661F771F0694A1F70590079420F4490FB5
:10521000561FC71FD81F990F661F771F881F069438
:10522000A9F784911095177041F0D695C7955795B9
:105230004795F794E7941A95C1F7EFE6F2E0689482
:105240001590159135916591959105907FE2739533
:10525000E118F10A430B560BC90BD009C0F7E10C5A
:10526000F11E431F561FC91FD01D7EF4703311F469
:105270008A95E6CFE894015030F0080F0AF4002731
:10528000021708F4202F2395022F7A3328F079E3B0
:105290007D932A95E9F710C07D932A9589F60694A7
:1052A00097956795379517951794E118F10A430B71
:1052B000560BC90BD00998F023957E9173957A33DC
:1052C00008F070E37C932013B8F77E9170617D93B2
:1052D00030F0839571E37D9370E32A95E1F7112413
:1052E000EF90FF900F911F91CF91DF91992787FD4C
:1052F0009095089591110C947E2A803219F089506E
:105300008550C8F70895FB01DC014150504088F0FA
:105310008D9181341CF08B350CF4805E6591613485
:105320001CF06B350CF4605E861B611171F3990BF8
:105330000895881BFCCFDC01FC01672F7191772356
:10534000E1F7329704C07C916D9370836291AE1740
:10535000BF07C8F308950E94ED2908F481E008957D
:10536000E89409C097FB3EF49095809570956195FF
:105370007F4F8F4F9F4F9923A9F0F92F96E9BB27B5
:105380009395F695879577956795B795F111F8CF31
:10539000FAF4BB0F11F460FF1BC06F5F7F4F8F4F9C
:1053A0009F4F16C0882311F096E911C0772321F092
:1053B0009EE8872F762F05C0662371F096E8862F2A
:1053C00070E060E02AF09A95660F771F881FDAF781
:1053D000880F9695879597F90895990F0008550FAE
:1053E000AA0BE0E8FEEF16161706E807F907C0F06B
:1053F00012161306E407F50798F0621B730B840B73
:10540000950B39F40A2661F0232B242B252B21F44C
:1054100008950A2609F4A140A6958FEF811D811DEC
:1054200008950E94242A0C94982A0E948A2A38F00F
:105430000E94912A20F0952311F00C94812A0C945B
:10544000872A11240C94CC2A0E94A92A70F3959FD4
:10545000C1F3950F50E0551F629FF001729FBB276B
:10546000F00DB11D639FAA27F00DB11DAA1F649F07
:105470006627B00DA11D661F829F2227B00DA11DBA
:10548000621F739FB00DA11D621F839FA00D611D40
:10549000221F749F3327A00D611D231F849F600D61
:1054A000211D822F762F6A2F11249F5750409AF08A
:1054B000F1F088234AF0EE0FFF1FBB1F661F771F16
:1054C000881F91505040A9F79E3F510580F00C94E1
:1054D000812A0C94CC2A5F3FE4F3983ED4F386955E
:1054E00077956795B795F795E7959F5FC1F7FE2B81
:1054F000880F911D9695879597F908959927882784
:10550000089597F99F6780E870E060E008959FEF45
:1055100080EC089500240A9416161706180609064A
:10552000089500240A941216130614060506089519
:10553000092E0394000C11F4882352F0BB0F40F4A1
:10554000BF2B11F460FF04C06F5F7F4F8F4F9F4FE1
:10555000089557FD9058440F551F59F05F3F71F063
:105560004795880F97FB991F61F09F3F79F08795CA
:105570000895121613061406551FF2CF4695F1DF53
:1055800008C0161617061806991FF1CF86957105E3
:10559000610508940895E894BB2766277727CB0117
:1055A00097F90895F999FECF92BD81BDF89A992790
:1055B00080B50895262FF999FECF1FBA92BD81BDFF
:1055C00020BD0FB6F894FA9AF99A0FBE0196089585
:1055D000052E97FB1EF400940E94FF2A57FD07D06A
:1055E0000E941A2B07FC03D04EF40C94FF2A50950E
:1055F0004095309521953F4F4F4F5F4F08959095BF
:105600008095709561957F4F8F4F9F4F08950E94B1
:105610003C2BA59F900DB49F900DA49F800D911DD4
:1056200011240895B7FF0C94072B0E94072B821BAF
:10563000930B0895A1E21A2EAA1BBB1BFD010DC0FE
:10564000AA1FBB1FEE1FFF1FA217B307E407F50732
:1056500020F0A21BB30BE40BF50B661F771F881F0E
:10566000991F1A9469F760957095809590959B01A4
:10567000AC01BD01CF010895A29FB001B39FC0014D
:10568000A39F700D811D1124911DB29F700D811D6E
:105690001124911D08955058BB27AA270E94632BFF
:1056A0000C94982A0E948A2A38F00E94912A20F0AD
:1056B00039F49F3F19F426F40C94872A0EF4E095F0
:1056C000E7FB0C94812AE92F0E94A92A58F3BA1704
:1056D000620773078407950720F079F4A6F50C9408
:1056E000CB2A0EF4E0950B2EBA2FA02D0B01B90199
:1056F00090010C01CA01A0011124FF27591B99F048
:10570000593F50F4503E68F11A16F040A22F232F53
:10571000342F4427585FF3CF469537952795A795A3
:10572000F0405395C9F77EF41F16BA0B620B730B4A
:10573000840BBAF09150A1F0FF0FBB1F661F771FBB
:10574000881FC2F70EC0BA0F621F731F841F48F470
:10575000879577956795B795F7959E3F08F0B0CFF9
:105760009395880F08F09927EE0F979587950895E0
:105770000E948A2A60F080E891E009F49EEF0E947E
:10578000912A28F040E851E071F45EEF0CC00C94CF
:10579000872A0C94CB2AE92FE0780E94A92A40F3AB
:1057A000092E052AB1F3261737074807590738F09D
:1057B0000E2E07F8E02569F0E025E0640AC0EF63EB
:1057C00007F8009407FADB01B9019D01DC01CA0169
:1057D000AD01EF930E94412C0E94982A0E94FB2B5E
:1057E0005F91552339F02BED3FE049E450FD49EC42
:1057F0000C944C2B0895DF93DD27B92FBF7740E839
:105800005FE31616170648075B0718F4D92F0E94A6
:10581000FE2C9F938F937F936F930E949C2DE4EEB9
:10582000F0E00E94D22C0E94982A2F913F914F9134
:105830005F910E94242ADD2351F09058A2EA2AEDBC
:105840003FE049EC5FE3D0785D270E94632BDF9156
:105850000C94982A0E943E2C0C94982A0E94912A1B
:1058600058F00E948A2A40F029F45F3F29F00C94F6
:10587000812A51110C94CC2A0C94872A0E94A92ABF
:1058800068F39923B1F3552391F3951B550BBB276F
:10589000AA2762177307840738F09F5F5F4F220FB4
:1058A000331F441FAA1FA9F335D00E2E3AF0E0E8AB
:1058B00032D091505040E695001CCAF72BD0FE2FF5
:1058C00029D0660F771F881FBB1F26173707480789
:1058D000AB07B0E809F0BB0B802DBF01FF27935841
:1058E0005F4F3AF09E3F510578F00C94812A0C945A
:1058F000CC2A5F3FE4F3983ED4F38695779567957D
:10590000B795F7959F5FC9F7880F911D9695879575
:1059100097F90895E1E0660F771F881FBB1F621794
:1059200073078407BA0720F0621B730B840BBA0B52
:10593000EE1F88F7E09508950E94A32C6894B1119A
:105940000C94CC2A08950E94B12A88F09F5798F0B1
:10595000B92F9927B751B0F0E1F0660F771F881F74
:10596000991F1AF0BA95C9F714C0B13091F00E948E
:10597000CB2AB1E008950C94CB2A672F782F882783
:10598000B85F39F0B93FCCF3869577956795B395B5
:10599000D9F73EF490958095709561957F4F8F4F24
:1059A0009F4F0895DF93CF931F930F93FF92EF9232
:1059B000DF927B018C01689406C0DA2EEF010E9411
:1059C000242AFE01E894A5912591359145915591A0
:1059D000A6F3EF010E94632BFE019701A801DA9460
:1059E00069F7DF90EF90FF900F911F91CF91DF91BA
:1059F00008950E94ED2908F48FEF08959B01AC01F2
:105A000060E070E080E89FE30C942A2CFA01EE0F2E
:105A1000FF1F309621053105A1F16115710561F473
:105A20008038BFE39B0749F168949038810561F0A5
:105A30008038BFEF9B0741F099234AF5FF3FE1050E
:105A40003105210519F1E8940894E795D901AA23B5
:105A500029F4AB2FBE2FF85FD0F310C0FF5F70F4B6
:105A6000A695E0F7F73950F019F0FF3A38F49F7730
:105A70009F930DD00F9007FC9058089546F00C941A
:105A8000872A60E070E080E89FE308954FE79F7702
:105A90005F934F933F932F930E94362E2F913F9108
:105AA0004F915F910E94112A0C94AD2D19F416F4B8
:105AB0000C94872A0C94DF2D0E94B12AB8F3992305
:105AC000C9F3B6F39F57550B87FF0E94ED2D0024B5
:105AD000A0E640EA900180585695979528F4805C9E
:105AE000660F771F881F20F026173707480730F406
:105AF000621B730B840B202931294A2BA69517941E
:105B00000794202531254A2758F7660F771F881FED
:105B100020F026173707480730F4620B730B840B0D
:105B2000200D311D411DA09581F7B901842F915899
:105B3000880F9695879508959B01AC010C94112AC6
:105B40000E94ED29880B990B089529F416F00C9406
:105B5000812A0C94CB2A0C94872A0E94B12AA8F39C
:105B60009638A0F707F80F92E8942BE33AEA48EB4F
:105B70005FE70E94272A0F920F920F924DB75EB7F0
:105B80000F920E947E2EE1E1F1E00E94D22C4F9113
:105B90005F91EF91FF91E595EE1FFF1F49F0FE57D2
:105BA000E0684427EE0F441FFA95E1F74195550B45
:105BB0000E94F82D0F9007FE0C94FE2C08959F3F35
:105BC00031F0915020F4879577956795B795880FB8
:105BD000911D9695879597F9089591505040660FBD
:105BE000771F881FD2F708950C94812A0C94DF2D1B
:105BF0000E94B12AD8F39923C9F3940F511DA3F33E
:105C00009150504094F059F0882332F0660F771F7E
:105C1000881F91505040C1F79E3F51052CF7880FC7
:105C2000911D9695879597F908955F3FACF0983E42
:105C30009CF0BB27869577956795B79508F4B1607A
:105C40009395C1F7BB0F58F711F460FFE8CF6F5F72
:105C50007F4F8F4F9F4FE3CF0C94CC2A16F00C94BC
:105C6000DF2D0C94872A68940C94812A0E94B12A13
:105C7000A8F39923C1F3AEF3DF93CF931F930F9350
:105C8000FF92C92FDD2788232AF02197660F771FFF
:105C9000881FDAF720E030E040E85FEB9FE38839C7
:105CA00020F0803E38F021968F770E944C2BE9E35C
:105CB000F1E004C00E944C2BE6E6F1E00E94D22CF9
:105CC0008B01BE01EC01FB2E6F5771097595771F93
:105CD000880B990B0E94B22928E132E741E35FE388
:105CE0000E94242AAF2D9801AE01FF900F911F91C1
:105CF000CF91DF910E94632B0C94982AFA01DC016A
:105D0000AA0FBB1F9B01AC01BF5728F422273327E2
:105D10004427507820C0B75190F4AB2F002446950B
:105D200037952795011CA395D2F3002071F0220F1F
:105D3000331F441FB395DAF30ED00C944B2B613014
:105D40007105A0E88A07B94630F49B01AC016627CB
:105D5000772788279078309621F0208331834283FB
:105D600053830895DB018F939F930E94072BBF916C
:105D7000AF91A29F800D911DA39F900DB29F900D9A
:105D800011240895AA1BBB1B51E107C0AA1FBB1F0A
:105D9000A617B70710F0A61BB70B881F991F5A95B7
:105DA000A9F780959095BC01CD010895EE0FFF1FD6
:105DB000881F8BBF0790F691E02D19940F931F93C6
:105DC000CF93DF938230910510F482E090E0E09170
:105DD0005E05F0915F0530E020E0B0E0A0E0309794
:105DE00099F42115310509F44AC0281B390B2430D8
:105DF0003105D8F58A819B816115710589F1FB0117
:105E000093838283FE0111C04081518102811381FD
:105E100048175907E0F04817590799F4109761F0AF
:105E200012960C93129713961C933296CF01DF9122
:105E3000CF911F910F91089500935E0510935F0518
:105E4000F4CF2115310551F04217530738F0A9015D
:105E5000DB019A01BD01DF01F801C1CFEF01F9CFEC
:105E600090935F0580935E05CDCFFE01E20FF31F97
:105E7000819391932250310939832883D7CF209180
:105E80005C0530915D05232B41F42091180230917F
:105E9000190230935D0520935C0520911602309124
:105EA00017022115310541F42DB73EB740911A0272
:105EB00050911B02241B350BE0915C05F0915D05B0
:105EC000E217F307A0F42E1B3F0B2817390778F0D1
:105ED000AC014E5F5F4F2417350748F04E0F5F1F30
:105EE00050935D0540935C05819391939FCFF0E0C3
:105EF000E0E09CCFCF93DF930097E9F0FC0132976D
:105F000013821282A0915E05B0915F05ED0130E031
:105F100020E01097A1F420813181820F931F2091FE
:105F20005C0530915D052817390709F061C0F093D1
:105F30005D05E0935C05DF91CF910895EA01CE17EE
:105F4000DF07E8F54A815B819E0141155105B1F7F4
:105F5000E901FB83EA8349915991C40FD51FEC17DE
:105F6000FD0761F4808191810296840F951FE901FC
:105F700099838883828193819B838A83F0E0E0E028
:105F800012968D919C9113970097B9F52D913C91A4
:105F90001197CD010296820F931F20915C053091DD
:105FA0005D052817390739F6309751F510925F05CE
:105FB00010925E05B0935D05A0935C05BCCFD383C2
:105FC000C28340815181840F951FC817D90761F49E
:105FD0004E5F5F4F88819981480F591F51834083DD
:105FE0008A819B81938382832115310509F0B0CF8B
:105FF000F0935F05E0935E059ECFFD01DC01C0CF0D
:1060000013821282D7CF4F925F926F927F928F92BC
:106010009F92AF92BF92CF92DF92EF92FF920F9337
:106020001F93CF93DF938C01009799F4CB01DF91FD
:10603000CF911F910F91FF90EF90DF90CF90BF9085
:10604000AF909F908F907F906F905F904F900C9447
:10605000DE2EFC01E60FF71F9C0122503109E217EA
:10606000F30708F4AEC0D901CD91DC911197C617A2
:10607000D70720F1C530D10578F0CE0104978617F7
:10608000970750F0C61BD70B2297C193D1936D93FE
:106090007C93CF010E947A2FC801DF91CF911F918D
:1060A0000F91FF90EF90DF90CF90BF90AF909F90B7
:1060B0008F907F906F905F904F9008955B01AC1A26
:1060C000BD0A4C018C0E9D1EA0915E05B0915F052E
:1060D000512C412CF12CE12C109731F580915C056D
:1060E00090915D058815990509F05CC04616570624
:1060F00008F058C08091160290911702009741F461
:106100008DB79EB740911A0250911B02841B950BCC
:10611000E817F90708F055C0F0935D05E0935C05BA
:10612000F90171836083B8CF8D919C91119712967C
:106130006C90129713967C901397A815B90559F592
:106140006C0142E0C40ED11CCA14DB0420F1AC0186
:106150004A195B09DA011296159780F06282738200
:1061600051834083D9016D937C93E114F10471F064
:10617000D7011396FC93EE9312978ECF22968C0F35
:106180009D1FF90191838083F301EFCFF0935F05A9
:10619000E0935E0581CF4816590608F42C017D0175
:1061A000D3019ACFCB010E94DE2E7C01009749F0EB
:1061B000AE01B8010E94EC30C8010E947A2F87011D
:1061C0006BCF10E000E068CF9111089581568A519D
:1061D00008F4805285580895FB01DC0102C001904B
:1061E0000D9241505040D8F70895FB01DC01019019
:1061F0000D920020E1F70895FB01DC014150504071
:1062000030F08D910190801919F40020B9F7881BA6
:10621000990B0895FB01DC014150504048F001907A
:106220000D920020C9F701C01D9241505040E0F787
:10623000089512E0C3EBD2E000E006C0802FFE011B
:106240000E94D62E2196011DC43BD10780E008078D
:06625000A9F7F894FFCF4E
:10625600000075440080894401640016000000A017
:10626600400000F0410100006005800000000000D1
:10627600CB031A036203180493037103850300001A
:1062860000002709FA086809EA08AF06E702EB08E2
:1062960000000000AE06450CB6064F1002100D0AAF
:1062A60000543D006F432000483D002500484D4303
:1062B6003538383300436F6D706173733A200028A8
:1062C6006465672920004E200045005320005700D2
:1062D600732000296D4700203D3E006F4320413D5D
:1062E600006D00496E636C2E20616E672E28782043
:1062F60079207A292F6465673A2000613D0020677E
:1063060000414E4D4C3033004E616E6F4132643564
:106316000073657269616C3A20002D35002D3400DA
:106326002D33002D32002D310044005665727369FD
:106336006F6E3A200023007300534C20503D0050EE
:106346006120697320756E6C696B656C79210053E9
:106356006561206C6576656C20503D002068506153
:066366000055565A00002C
:00000001FF
